:020000040000FA
:1000000015EF00F0FFFFFFFF04EF14F01200FFFFF9
:10001000FFFFFFFFFFFFFFFF64EF00F01200FFFF95
:10002000FFFFFFFFFFFFFFFFFFFF0001000EE16E7C
:10003000E26E000EE66EE2500808FBE160EF00F0B1
:10004000FFFFFFFFFFFFFFFFFFFFFFFFFFFFFFFFC0
:10005000FFFFFFFFFFFFFFFFFFFFFFFFFFFFFFFFB0
:10006000FFFFFFFFFFFFFFFFFFFFFFFFFFFFFFFFA0
:10007000FFFFFFFFFFFFFFFFFFFFFFFFFFFFFFFF90
:100080004D43485000FFFFFFFFFFFFFFFFFFFFFF53
:10009000FFFFFFFFFFFFFFFFFFFFFFFFFFFFFFFF70
:1000A000FFFFFFFFFFFFFFFFFFFFFFFFFFFFFFFF60
:1000B000FFFFFFFFFFFFFFFFFFFFFFFFFFFFFFFF50
:1000C00054EF10F01200FFFF34EF10F01200FFFFAA
:1000D0008201FFFFFFFFFFFFFFFFFFFFFFFFFFFFAB
:1000E000CC02DA02E202FFFFFFFFFFFFFFFFFFFF8C
:1000F000FFFFFFFFFFFFFFFFFFFFFFFFFFFFFFFF10
:100100000200C42000004000000010000000C020D9
:1001100000005A00000004000000D9CFE6FFE1CF44
:10012000D9FF020EE1268F0EDE6E000EDD6EDECFF1
:10013000E9FFDDCFEAFF010EEE6EED6AD00EF66E3E
:10014000000EF76E0900F5CF10F00800F5CF11F0A2
:10015000DECFE9FFDDCFEAFF020EE926000EEA223C
:1001600010C0EEFF11C0EDFF8F0EE66E000EE66EC2
:1001700020EC07F0E552E552F56E020EE15C02E27A
:10018000E16AE552E16EF550E552E7CFD9FF120082
:10019000D9CFE6FFE1CFD9FFE652F19E89D8DF6ED5
:1001A0000001F05107E1DF5005E12DD8000902E020
:1001B00000EF14F0E66A01EC08F0E552DDEC07F020
:1001C000140E6F6E0001976B0001986B0001996B24
:1001D00080A802D0ECEC07F035EC0AF051EC0AF004
:1001E00000090BE0080EE66E400EE66E000EE66EAD
:1001F00081EC01F0E552E552E552EAD7E552E552CD
:10020000E7CFD9FF1200D9CFE6FFE1CFD9FF060E25
:10021000E126DE6A280EDD6E040EDB6A050EDB6A5F
:10022000020EDB6A030EDB6A040EDBCF10F0050E54
:10023000DBCF11F0000E105C2C0E115821E2D9CF4B
:10024000E9FFDACFEAFFEECFF6FFEDCFF7FF020EC0
:10025000EE26000EEF220900F5CF10F00800F5CFD2
:1002600011F0D950020FE96EDACFEAFF1050EE26F6
:100270001150ED22040EDB2A050E01E3DB2AD4D750
:10028000D950020FE96EDACFEAFFEE50ED1002E02E
:10029000000E01D0010EF56E060EE15C03E200D007
:1002A000E16AE552E16EF550E552E7CFD9FF120061
:1002B000938E8150800B02E0000E01D0010E00D021
:1002C0001200F29CF29ED59E6D6A12000001010E92
:1002D000F06FF7DF60EF00F01200F3DF00EF00F0E7
:1002E0001200D00EF66E000EF76E0900F5CF10F07A
:1002F0000800F5CF11F010C0F3FF11C0F4FF00D0DB
:100300001200D9CFE6FFE1CFD9FF120EE66E7D0EC7
:10031000E66E000EE66EBDEC06F0E552E552E552E3
:10032000FC0EDB500001D8807D551FE3FD0EDBCFB6
:1003300012F0FE0EDBCF13F07D51020D1250F324AC
:10034000E96E1350F420EA6EEECF10F0EFCF11F00B
:100350007D0EE66E000EE66E04D011C0FAFF10505E
:10036000F96EFBDFE552E55210D00001010E8F6FF0
:10037000906B916B926B936B946B8F0EE66E000E8D
:10038000E66E20EC07F0E552E55200017D69E5528A
:10039000E7CFD9FF1200D9CFE6FFE1CFD9FF0E0E8C
:1003A000E126FD0EDBCFE9FFFE0EDBCFEAFF020EFA
:1003B000E926000EEA22EECF04F0EECF05F0EECFF4
:1003C00006F0EFCF07F0400E096E0A6A0B6A0C6A5E
:1003D00010EC10F004C0DEFF05C0DDFFFD0EDBCF2A
:1003E000E9FFFE0EDBCFEAFF020EE926000EEA224D
:1003F000EECF04F0EECF05F0EECF06F0EFCF07F032
:10040000400E096E0A6A0B6A0C6A10EC10F0020EBC
:1004100000C0DBFFFD0EDBCFE9FFFE0EDBCFEAFF06
:10042000020EE926000EEA22080EE926000EEA2254
:10043000030EEECFDBFF040EEECFDBFF050EEECF9B
:10044000DBFF060EEECFDBFF0B0EDB6A0C0EDB6A6A
:100450000D0EDB6A070EDB6A080EDB6A070EDBCFC8
:1004600010F0080EDBCF11F0DECF12F0DDCF13F06D
:100470001250105C1350115848E2D950090FE66E23
:10048000000EDA20E66ED950030FE96EDACFEAFFEC
:10049000EECFE6FFEECFE6FFEECFE6FFEFCFE6FFD3
:1004A000400EE66EE66A800EE66E050EE66E78ECAD
:1004B00009F0F56E0A0EE15EF550E76E0D0EE7CF1E
:1004C000DBFF090EDBCF10F00A0EDBCF11F0D950A5
:1004D0000B0FE96EDACFEAFF1050EE261150ED2235
:1004E000090EDBCFE6FF000EE66EE66AE9EC06F0E9
:1004F000E552E552E5520D0EDB5001E006D0070E45
:10050000DB2A080E01E3DB2AA9D7020EDB5042E00A
:100510000D0EDB503FE1D950090FE66E000EDA20D8
:10052000E66ED950030FE96EDACFEAFFEECFE6FFB1
:10053000EECFE6FFEECFE6FFEFCFE6FF020EDBCF1A
:10054000E6FFE66A800EE66E050EE66E78EC09F0D0
:10055000F56E0A0EE15EF550E76E0D0EE7CFDBFF9C
:10056000090EDBCF10F00A0EDBCF11F0D9500B0FC4
:10057000E96EDACFEAFF1050EE261150ED22090E97
:10058000DBCFE6FF000EE66EE66AE9EC06F0E55228
:10059000E552E5520D0EDB5007E100018F6B906BC9
:1005A000916B926B936B0BD00001020E8F6F0B0E51
:1005B000DBCF90F00C0EDBCF91F0926B936B906BD6
:1005C000916B926B936B946B8F0EE66E000EE66EE2
:1005D00020EC07F0E552E552F56E0E0EE15C02E20A
:1005E000E16AE552E16EF550E552E7CFD9FF12001E
:1005F000D9CFE6FFE1CFD9FF0E0EE126FD0EDBCF0E
:10060000E9FFFE0EDBCFEAFF020EE926000EEA222A
:10061000EECF04F0EECF05F0EECF06F0EFCF07F00F
:10062000400E096E0A6A0B6A0C6A10EC10F004C0E6
:10063000DEFF05C0DDFFFD0EDBCFE9FFFE0EDBCFE9
:10064000EAFF020EE926000EEA22EECF04F0EECF1A
:1006500005F0EECF06F0EFCF07F0400E096E0A6A04
:100660000B6A0C6A10EC10F0020E00C0DBFFFD0EEE
:10067000DBCFE9FFFE0EDBCFEAFF020EE926000E1C
:10068000EA22080EE926000EEA22030EEECFDBFF77
:10069000040EEECFDBFF050EEECFDBFF060EEECF36
:1006A000DBFF0B0EDB6A0C0EDB6A0D0EDB6A070E3E
:1006B000DB6A080EDB6A070EDBCF10F0080EDBCF1B
:1006C00011F0DECF12F0DDCF13F01250105C13509A
:1006D00011584EE2E66AE66A010EE66E89EC07F012
:1006E000E552E552E552D950090FE66E000EDA20C8
:1006F000E66ED950030FE96EDACFEAFFEECFE6FFE0
:10070000EECFE6FFEECFE6FFEFCFE6FF400EE66E60
:10071000E66A000EE66E050EE66EBDEC08F0F56EBC
:100720000A0EE15EF550E76E0D0EE7CFDBFF090E16
:10073000DBCF10F00A0EDBCF11F0D9500B0FE96EB2
:10074000DACFEAFF1050EE261150ED22E66A000ED5
:10075000E66EE66A12DBE552E552E5520D0EDB501D
:1007600001E006D0070EDB2A080E01E3DB2AA3D73F
:10077000020EDB5047E00D0EDB5044E1E66AE66A0C
:10078000010EE66EC6DBE552E552E552D950090F7F
:10079000E66E000EDA20E66ED950030FE96EDACF6E
:1007A000EAFFEECFE6FFEECFE6FFEECFE6FFEFCFBC
:1007B000E6FF020EDBCFE6FFE66A000EE66E050EF0
:1007C000E66EBDEC08F0F56E0A0EE15EF550E76EE0
:1007D0000D0EE7CFDBFF090EDBCF10F00A0EDBCFEB
:1007E00011F0D9500B0FE96EDACFEAFF1050EE2668
:1007F0001150ED22E66A000EE66EE66ABEDAE552B8
:10080000E552E5520D0EDB5007E100018F6B906B56
:10081000916B926B936B0BD00001010E8F6F0B0EDF
:10082000DBCF90F00C0EDBCF91F0926B936B946B5F
:100830008F0EE66E000EE66E03DBE552E552F56EB6
:100840000E0EE15C02E2E16AE552E16EF550E5521E
:10085000E7CFD9FF1200D9CFE6FFE1CFD9FF97EC60
:1008600008F000018F6B906B916B926B936B946BA4
:100870008F0EE66E000EE66EE3DAE552E552E552C3
:10088000E7CFD9FF1200D9CFE6FFE1CFD9FF020EA3
:10089000E1268F0EDE6E000EDD6EF29E5CC0F6FF6E
:1008A0005DC0F7FF0900F5CF10F00800F5CF11F09B
:1008B000DECFE9FFDDCFEAFF10C0EEFF11C0EDFF94
:1008C000F28E8F0EE66E000EE66EBADAE552E55253
:1008D000F56E020EE15C02E2E16AE552E16EF5506E
:1008E000E552E7CFD9FF1200D9CFE6FFE1CFD9FF1C
:1008F000090EE12600018F6BFD0EDBCFE9FFFE0E36
:10090000DBCFEAFF020EE926000EEA22EECF10F05E
:10091000EFCF11F0010E101801E1115001E102D1E9
:10092000020E101801E1115049E0105001E1115080
:1009300001E0F8D0FD0EDBCFE9FFFE0EDBCFEAFFD2
:10094000020EE926000EEA22040EE926000EEA2233
:10095000EECF10F0EFCF11F0060ED890113210321A
:10096000E804FBE110C0DEFF11C0DDFFD9CFE9FFD5
:10097000DACFEAFFEE50ED101DE0DECFE6FFDDCF6F
:10098000E6FFFD0EDBCFE9FFFE0EDBCFEAFF020E36
:10099000E926000EEA22020EE926000EEA22EECF38
:1009A000E6FFEFCFE6FF93EC0EF0E552E552E5529D
:1009B000E55203D00001040E8F6F5CD1FD0EDBCF3A
:1009C000E9FFFE0EDBCFEAFF020EE926000EEA2267
:1009D000040EE926000EEA22EECF10F0EFCF11F060
:1009E000060E0F0B05E0D89011321032E806FBE13D
:1009F000040E10C0DBFF050E11C0DBFFFD0EDBCFC8
:100A0000E9FFFE0EDBCFEAFF020EE926000EEA2226
:100A1000040EE926000EEA22EECF10F0EFCF11F01F
:100A20000001116A3F0E1016080E10C0DBFFFD0E0C
:100A3000DBCFE9FFFE0EDBCFEAFF020EE926000E58
:100A4000EA22020EE926000EEA22060EEECFDBFFB6
:100A5000070EEDCFDBFF020EDB6A030EDB6A020E30
:100A6000DBCF10F0030EDBCF11F0040EDBCF12F062
:100A7000050EDBCF13F01250105C135011582EE20C
:100A8000E66AE66A010EE66E44DAE552E552E552A0
:100A9000000EE66E050EE66E060EDBCFE6FF070ED5
:100AA000DBCFE6FFCBEC0EF0E552E552E552E55226
:100AB000D950060FE96EDACFEAFF400EEE26000E9F
:100AC000ED22E66AE66EE66A58D9E552E552E5524D
:100AD000020EDB2A030E01E3DB2AC1D7080EDB502E
:100AE00020E0E66AE66A010EE66E13DAE552E552A8
:100AF000E552000EE66E050EE66E060EDBCFE6FF53
:100B0000070EDBCFE6FFCBEC0EF0E552E552E552E7
:100B1000E552E66A000EE66EE66A2FD9E552E55226
:100B2000E552A8D0FD0EDBCFE9FFFE0EDBCFEAFFDA
:100B3000020EE926000EEA22040EE926000EEA2241
:100B4000EECF10F0EFCF11F0060E0F0B05E0D890AE
:100B500011321032E806FBE1040E10C0DBFF050E77
:100B600011C0DBFFFD0EDBCFE9FFFE0EDBCFEAFF9E
:100B7000020EE926000EEA22040EE926000EEA2201
:100B8000EECF10F0EFCF11F00001116A3F0E1016FA
:100B9000080E10C0DBFFFD0EDBCFE9FFFE0EDBCF42
:100BA000EAFF020EE926000EEA22020EE926000EF6
:100BB000EA22060EEECFDBFF070EEDCFDBFF020EC3
:100BC000DB6A030EDB6A020EDBCF10F0030EDBCF15
:100BD00011F0040EDBCF12F0050EDBCF13F0125034
:100BE000105C1350115828E2800EE66E050EE66E7A
:100BF000060EDBCFE6FF070EDBCFE6FF21EC0FF0A2
:100C0000E552E552E552E552D950060FE96EDACFCA
:100C1000EAFF400EEE26000EED22400EE66E000EBC
:100C2000E66EE66AD6D8E552E552E552020EDB2AB8
:100C3000030E01E3DB2AC7D7080EDB501AE0800E53
:100C4000E66E050EE66E060EDBCFE6FF070EDBCF87
:100C5000E6FF21EC0FF0E552E552E552E552080EB1
:100C6000DBCFE6FF000EE66EE66AB3D8E552E5524A
:100C7000E55200D00001906B916B926B936B946B7B
:100C80008F0EE66E000EE66EDBD8E552E552F56E8D
:100C9000090EE15C02E2E16AE552E16EF550E552CF
:100CA000E7CFD9FF1200D9CFE6FFE1CFD9FF00018E
:100CB0008F6B906B916B926B936B946B8F0EE66E58
:100CC000000EE66EBDD8E552E552C80EE66EE66A45
:100CD000E66AE66A49EC08F0E552E552E552E5526B
:100CE0006D96F29E5AC0F6FF5BC0F7FF020EF62625
:100CF000000EF7220900F5CF10F00800F5CF11F033
:100D000004D011C0FAFF1050F96EFBDFE552E7CFB7
:100D1000D9FF1200D9CFE6FFE1CFD9FF00018F6BD9
:100D2000906B916B926B936B946B8F0EE66E000ED3
:100D3000E66E86D8E552E552C80EE66EE66AE66AC9
:100D4000E66A49EC08F0E552E552E552E5526D9647
:100D5000F29E5AC0F6FF5BC0F7FF0900F5CF10F016
:100D60000800F5CF11F004D011C0FAFF1050F96E51
:100D7000FBDFE552E7CFD9FF1200D9CFE6FFE1CF85
:100D8000D9FFD950FD0FE96EFF0EDA20EA6EEE5062
:100D9000ED1013E0FC0EDBCFE6FFE66A000EE66E18
:100DA000050EE66EFD0EDBCFE6FFFE0EDBCFE6FFA7
:100DB000D8D8F56E060EE15EF55068960401400E37
:100DC000096F0817087D880E0813E552E7CFD9FF91
:100DD0001200D9CFE6FFE1CFD9FFD950FD0FE96E60
:100DE000FF0EDA20EA6EEE50ED1013E0FC0EDBCFC2
:100DF000E6FFE66AFD0EDBCFE6FFFE0EDBCFE6FF89
:100E0000800EE66E050EE66EACD8F56E060EE15E5F
:100E1000F550FC0EDBCF15F4400E04011417147DC1
:100E2000880E1413010EE66E040EE66E020EE66ED8
:100E300070D8E552E552E552E552E7CFD9FF1200EE
:100E4000D9CFE6FFE1CFD9FF050EE1260EC4DEFFC4
:100E50000FC4DDFFFD0EDBCF06F0FE0EDBCF07F08B
:100E6000020E06C0DBFF030E07C0DBFF080EF36EA9
:100E7000040EF3CFDBFFDBCF0DF4DFCFE9FFDF2A7A
:100E8000010EDBCFEAFF01E3DB2A7DC0EFFFDFCFFE
:100E9000E9FFDF2ADBCFEAFF01E3DB2AEF6A040E7A
:100EA000DBCFF3FFDB06F350000917E0020EDBCFC8
:100EB000E9FFDB2A030EDBCFEAFF01E3DB2AEF5079
:100EC000E66EDFCFE9FFDF2A010EDBCFEAFF01E3A9
:100ED000DB2AE552E750EF6EE2D7400E04010C1713
:100EE0000C7D880E0C13010EE66E040EE66E010EEC
:100EF000E66E0FD8E552E552E552F56E050EE15C5F
:100F000002E2E16AE552E16EF550E552E7CFD9FF22
:100F10001200D9CFE6FFE1CFD9FF35EC0AF051EC52
:100F20000AF0000919E0780E00017C15E840E8405D
:100F3000E8401F0B106EFE0EDB50105C0DE1040E3E
:100F40007C15116EFD0EDB50115C06E1FC0EDB50D2
:100F500001E0689602D000D0E0D7E552E7CFD9FF94
:100F60001200D9CFE6FFE1CFD9FFF90EDBCF10F0A9
:100F7000DB06FA0EDBCF11F001E2DB061050111098
:100F800018E0FB0EDBCFE9FFDB2AFC0EDBCFEAFF2C
:100F900001E3DB2AEF50E66EFD0EDBCFE9FFDB2A33
:100FA000FE0EDBCFEAFF01E3DB2AE552E750EF6EEE
:100FB000DCD7E552E7CFD9FF12000F0EC16E070E46
:100FC000B46E8B8494948B92949280807E0E926EF9
:100FD00089EF08F06D961200BBEC08F0FBDF8BA2E6
:100FE00002D08B9201D08B82140EE66EE66AE66A1E
:100FF000E66A49EC08F0E552E552E552E552EFD7D2
:101000001200D9CFE6FFE1CFD9FF0001706B716B01
:10101000726B736BD56AD08EFE0EDB5002E0F184EA
:1010200001D0F194150ED76EA00ED66EF294F28A0E
:10103000F28CF28ED58EE552E7CFD9FF1200D9CFD0
:10104000E6FFE1CFD9FF040EE126F29A70C0DFFF80
:10105000010E71C0DBFF020E72C0DBFF030E73C016
:10106000DBFFF28ADECF04F0DECF05F0DECF06F044
:10107000DDCF07F0DD52DD52F56E040EE15C03E2D8
:1010800000D0E16AE552E16EF550E552E7CFD9FFB5
:101090001200D9CFE6FFE1CFD9FF040EE12670C0E0
:1010A000DFFF010E71C0DBFF020E72C0DBFF030E1B
:1010B00073C0DBFFFB0EDBCF10F0FC0EDBCF11F0BB
:1010C000FD0EDBCF12F0FE0EDBCF13F0D9CFE9FF20
:1010D000DACFEAFFEE501026EE501122EE50122227
:1010E000EE50132210500001705D115071591250D2
:1010F00072591350735901E2DDD7F56E040EE15CAD
:1011000002E2E16AE552E16EF550E552E7CFD9FF20
:101110001200F18E470E836E956A8A888D808D82CB
:101120008A96E70E936EF90E946E966A1200D9CFE6
:10113000E6FFE1CFD9FF020EE1268A86DE6ADD6A8C
:10114000DECF10F0DDCF11F0480E105C920E11587A
:1011500005E2DF2A010E01E3DB2AF2D78A96F56E5B
:10116000020EE15C02E2E16AE552E16EF550E55201
:10117000E7CFD9FF12008A861200D9CFE6FFE1CF70
:10118000D9FF070EE126DF6AD950F70FE96EFF0E8F
:10119000DA20EA6E050EEE5C000EEE58000EEE58F8
:1011A000000EEE580BE2050EF36EF70EF3CFDBFFE9
:1011B000F80EDB6AF90EDB6AFA0EDB6A050EDB6AF3
:1011C000060EDB6A050EDBCF10F0060EDBCF11F04A
:1011D000FB0EDBCF12F0FC0EDBCF13F01250105CD5
:1011E000135011586BE21FEC08F0010E04C0DBFF36
:1011F000020E05C0DBFF030E06C0DBFF040E07C0B6
:10120000DBFF82B042D0010EDBCF14F0020EDBCF49
:1012100015F0030EDBCF16F0040EDBCF17F014C071
:10122000E6FF15C0E6FF16C0E6FF17C0E6FF1FEC9D
:1012300008F0E552E7CF17F0E552E7CF16F0E55298
:10124000E7CF15F0E552E7CF14F000011450045C2D
:10125000106E15500558116E16500658126E175024
:101260000758136ED950F70FE96EFF0EDA20EA6EB9
:101270001050EE5C1150EE581250EE581350EE58CC
:1012800003E2010EDF6E01D0BCD7DF0402E116D00D
:101290000FD08A988D90FD0EDBCFE9FFDB2AFE0E82
:1012A000DBCFEAFF01E3DB2AEF50836E8D808A8873
:1012B000050EDB2A060E01E3DB2A84D7F50EDBCF11
:1012C000E9FFF60EDBCFEAFF050EDBCFEEFF060EE1
:1012D000DBCFEDFFDF50F56E070EE15C03E200D0DF
:1012E000E16AE552E16EF550E552E7CFD9FF120011
:1012F000D9CFE6FFE1CFD9FF070EE126DF6AD9504B
:10130000F70FE96EFF0EDA20EA6E050EEE5C000EB6
:10131000EE58000EEE58000EEE580BE2050EF36E7E
:10132000F70EF3CFDBFFF80EDB6AF90EDB6AFA0E7D
:10133000DB6A050EDB6A060EDB6A050EDBCF10F0FA
:10134000060EDBCF11F0FB0EDBCF12F0FC0EDBCF75
:1013500013F01250105C135011586DE21FEC08F09E
:10136000010E04C0DBFF020E05C0DBFF030E06C04A
:10137000DBFF040E07C0DBFF82B042D0010EDBCFE3
:1013800014F0020EDBCF15F0030EDBCF16F0040EC7
:10139000DBCF17F014C0E6FF15C0E6FF16C0E6FF6E
:1013A00017C0E6FF1FEC08F0E552E7CF17F0E55253
:1013B000E7CF16F0E552E7CF15F0E552E7CF14F08E
:1013C00000011450045C106E15500558116E165033
:1013D0000658126E17500758136ED950F70FE96E62
:1013E000FF0EDA20EA6E1050EE5C1150EE581250EB
:1013F000EE581350EE5803E2010EDF6E01D0BCD759
:10140000DF0402E118D011D095688A988D928D8200
:10141000FD0EDBCFE9FFDB2AFE0EDBCFEAFF01E3A7
:10142000DB2A83CFEFFF8A88956A050EDB2A060E3A
:1014300001E3DB2A82D7F50EDBCFE9FFF60EDBCF27
:10144000EAFF050EDBCFEEFF060EDBCFEDFFDF5030
:10145000F56E070EE15C03E200D0E16AE552E16E51
:10146000F550E552E7CFD9FF12006DA60CD8000168
:10147000970508E16DBA06D0686A696A698069886B
:10148000020E976F12006D6A696A6D860001010E87
:10149000976F12006D6A696A0001976B12004AEF3C
:1014A0000AF0D9CFE6FFE1CFD9FF020EE126010E07
:1014B000DB6A0001975101E152D06850040B04E04F
:1014C0006950040B01E05ED86DB249D06850010B41
:1014D00004E06950010B01E078D86850100B04E07B
:1014E0006950100B01E04AD86850400B04E0695085
:1014F000400B01E05DD86850200B04E06950200BE0
:1015000001E058D86850020B04E06950020B01E07A
:101510005AD8030E0001975D01E221D06850080BF4
:101520001CE06950080B19E093EC0BF0F3CF10F0BE
:10153000F4CF11F0105011100FE16C50DF6EDFCFBF
:101540007CF0780EDF14E840E840E8401F0BE76EBF
:10155000010EE7CFDBFF01D0689601D0AAD7010EBC
:10156000DB50F56E020EE15C03E200D0E16AE55269
:10157000E16EF550E552E7CFD9FF12006984689813
:101580006D8212006D92699468941200000198A116
:101590000ED0F8DF6D840001080E956F070E966F70
:1015A0009507000E965B95519611FAE16D94120025
:1015B000689C1200010E7014010803E101EC0DF0AB
:1015C0007090689A1200689212006A6A686A9F0EA8
:1015D0006B6E7B0E696E6E6A0F0EE66E710EE66EB6
:1015E0000F0EE66E14D8E552E552E552160E706EF7
:1015F00068A602D06896FCD76D9801EC0DF000014A
:1016000098910001996B0001030E976F1200D9CFDA
:10161000E6FFE1CFD9FFFD0EDBCFE9FFFE0EDBCF0A
:10162000EAFFFC0EDB5004E0EE6AFC0EDB06F9D7A5
:10163000E552E7CFD9FF1200040140511F0B01080A
:1016400001E011D04051600BE842E842E842E84234
:10165000E842020801E007D0445101E004D04151C2
:1016600001E001D000D0120000017D690401400EAC
:10167000096F000E0A6F050E0B6F800E086F0401D4
:10168000400E0D6F400E0E6F050E0F6F400E0C6F6B
:101690000401126B136B800E106F0401400E156F66
:1016A000800E166F050E176F400E146F04011A6B33
:1016B0001B6B800E186F04011E6B1F6B400E1C6F9E
:1016C0000401226B236B800E206F0401266B276BB5
:1016D000400E246F04012A6B2B6B800E286F0401CF
:1016E0002E6B2F6B400E2C6F0401326B336B800E10
:1016F000306F0401366B376B400E346F04013A6B68
:101700003B6B800E386F04013E6B3F6B400E3C6FAD
:101710001E0E716E1A0E726E180E736E746E756EEA
:10172000766E776E1200D9CFE6FFE1CFD9FF020EB9
:10173000E126010EDE6EDD6A6C500BE10401005102
:101740003C0BE842E8420D0802E11FD801D031D835
:1017500007D0040E6C5C02E13CD802D0DE6ADD6A80
:10176000DECF10F0DDCF11F010C0F3FF11C0F4FF99
:10177000F56E020EE15C03E200D0E16AE552E16E33
:10178000F550E552E7CFD9FF1200D9CFE6FFE1CF00
:10179000D9FFE6520001746B0001756B00017A6B92
:1017A0007B6B0FEC0DF0E7D8E552E552E7CFD9FFA0
:1017B0001200020E0001745D0AE19BD8040100BD15
:1017C00003D0C80E006F02D0880E006F01D019D967
:1017D0001200040E0001975D0AE142C46EFF6E50D4
:1017E000000803E2050E976F02D0030E976F000109
:1017F00074050AE10BD8040104BD03D0C80E046FC0
:1018000002D0880E046F01D0FCD81200D9CFE6FFB9
:10181000E1CFD9FF020EE1260001080E7A5D000E2D
:101820007B5905E27AC0DEFF7BC0DDFF03D0080EE6
:10183000DE6EDD6A040104930491010EDB50041393
:10184000DFCF05F4000EDB5000017A5F010EDB50A4
:101850007B5B0001480E786F040E796F000198A33E
:101860001FD0D9CFE9FFDACFEAFFEE50ED1017E035
:1018700076C0F6FF77C0F7FF0800F55078C0E9FFA3
:1018800079C0EAFFEF6E0001782B000E792300018A
:10189000762B7723DF06010E01E2DB06E2D71DD0AF
:1018A000D9CFE9FFDACFEAFFEE50ED1016E076C0AF
:1018B000E9FF77C0EAFFEF5078C0E9FF79C0EAFF9F
:1018C000EF6E0001782B000E79230001762B772331
:1018D000DF06010E01E2DB06E3D7F56E020EE15CE6
:1018E00002E2E16AE552E16EF550E552E7CFD9FF39
:1018F0001200D9CFE6FFE1CFD9FF020EE126030E99
:1019000004010015E76E010EE7CFDBFF01C4DFFF26
:10191000DE5000017A27DD507B230001480E766FF0
:10192000040E776FD9CFE9FFDACFEAFFEE50ED1062
:1019300016E076C0E9FF77C0EAFFEF5078C0E9FF14
:1019400079C0EAFFEF6E0001782B000E79230001C9
:10195000762B7723DF06010E01E2DB06E3D7F56E77
:10196000020EE15C02E2E16AE552E16EF550E552F9
:10197000E7CFD9FF1200000175510CE10401080EF8
:10198000016F400E026F040E036F840E006F04019E
:10199000046F35D0040140AF22D000017A51040118
:1019A000465D00017B510401475904E246C47AF0C8
:1019B00047C47BF02BDF0001010E746F0401080E99
:1019C000016F400E026F040E036F800E006F040162
:1019D000480E066F040E076FC80E046F10D000018A
:1019E000020E746F0401056BC80E046F0401080E2B
:1019F000016F480E026F040E036FC80E006F6D98E2
:101A000012000001746B0401080E016F400E026F9A
:101A1000040E036F880E006F0401046B12000401B2
:101A20004051600BE842E842E842E842E8420009DF
:101A300001E055D04151070A51E00B0A4FE0070A77
:101A400040E0010A2CE00B0A28E0020A26E0030A23
:101A500022E0080A12E0010A0EE00F0A0AE0030A77
:101A600001E03CD00001010E756F0001040E976F7C
:101A700036D036D834D090D832D00001010E756FF0
:101A80000001990E766F000E776F000198930001A8
:101A9000010E7A6F24D0A8D822D0F4D820D000012B
:101AA000010E756F040144510001766F776B9A0E39
:101AB0007627000E7723000198930001010E7A6FBC
:101AC0000ED00001010E756F04014451EA6A9A0FAD
:101AD000E96E000EEA2242C4EFFF01D000D01200EE
:101AE000800E0401405D57E14351030A34E0010ACE
:101AF00010E0030A01E04DD00001010E756F0001F6
:101B00008E0E766F1E0E776F120E00017A6F7B6B52
:101B100040D00001010E756F04014251F66EF76A64
:101B2000D890F636F736740EF6261F0EF722090007
:101B3000F5CF76F00A00F5CF77F0020E0001F76AD4
:101B40007625F66E7751F7220900F5CF7AF00A0074
:101B5000F5CF7BF01ED00001010E756F04014251DC
:101B6000F66EF76AD890F636F736780EF6261F0E20
:101B7000F7220900F5CF76F00A00F5CF77F076C0AE
:101B8000F6FF77C0F7FF0800F55000017A6F7B6B16
:101B900000D00001988312000001010E756F0F0E36
:101BA000E66E710EE66E0F0EE66E07EC0BF0E55278
:101BB000E552E552010EE66E9A0EE66E000EE66EF6
:101BC00007EC0BF0E552E552E55242C499F00401EE
:101BD000425104E10001050E976F05D00001060E89
:101BE000976F34EC0BF012000401486B496B040151
:101BF00040511F0B020A14E0030A0EE0010A01E043
:101C000033D00001010E756F04014881000198A1D5
:101C100002D00401488328D00001010E756F24D042
:101C20000001010E756F040144510F0B080DF350B4
:101C3000116A000F106E040E11224451800B01E056
:101C4000010E040DF35000011024786F000E1120D6
:101C5000796F78C0E9FF79C0EAFFEF50040B03E029
:101C60000401010E486F00D0000175050AE1000172
:101C7000480E766F040E776F000198930001020EF4
:101C80007A6F12000401420510E140511F0B000958
:101C90000CE10001010E756F030E0401415D03E1CB
:101CA0000001988102D000019891040142513AE16B
:101CB00040511F0B020836E144510F0B000932E07E
:101CC0000001010E756F040144510F0B080DF35014
:101CD000116A000F106E040E11224451800B01E0B6
:101CE000010E040DF35000011024786F000E112036
:101CF000796F030E0401415D07E1840E78C0E9FFAE
:101D000079C0EAFFEF6E0ED044AF06D078C0E9FF8D
:101D100079C0EAFFEF6A06D0880E78C0E9FF79C083
:101D2000EAFFEF6E1200D9CFE6FFE1CFD9FFFD0E3B
:101D3000DBCFF6FFFE0EDBCFF7FFF86AA68EA69C80
:101D4000A684A688F29E550EA76EAA0EA76EA6823E
:101D50000000A6B2A9EF0EF0F28EA694FB0EDB06F1
:101D6000FC0E01E2DB06D950FB0FE96EFF0EDA2014
:101D7000EA6EEE50ED100BE0D950FD0FE96EFF0E4C
:101D8000DA20EA6E400EEE26000EED22D0D7E552A4
:101D9000E7CFD9FF1200D9CFE6FFE1CFD9FF020E7E
:101DA000E126DE52020EDD6EFD0EDBCFF6FFFE0EEB
:101DB000DBCFF7FFF86A200EDF6EFB0EDBCFE9FF0B
:101DC000DB2AFC0EDBCFEAFF01E3DB2AEF50F56EE6
:101DD0000D00DF06DF50000801E2EFD7FD0EDBCF7C
:101DE000F6FFFE0EDBCFF7FFF86AA68EA69CA68450
:101DF000A698F29E550EA76EAA0EA76EA6820000A8
:101E0000A6B200EF0FF0F28EA694010EDB06010ED3
:101E1000DB500BE0D950FD0FE96EFF0EDA20EA6EC1
:101E2000200EEE26000EED22BFD7F56E020EE15C0D
:101E300002E2E16AE552E16EF550E552E7CFD9FFE3
:101E40001200D9CFE6FFE1CFD9FFE652400EDF6E98
:101E5000FD0EDBCFF6FFFE0EDBCFF7FFF86A0900C1
:101E6000FB0EDBCFE9FFFC0EDBCFEAFFF5CFEFFF88
:101E7000FB0EDB2AFC0E01E3DB2ADF06DF50000845
:101E800001E2EDD7E552E552E7CFD9FF120012018A
:101E90000001FFFFFF08D8040180100000000001CE
:101EA000090274000101008032090400000EFFFFE6
:101EB000FF00070501024000000705020240000084
:101EC0000705030240000007050402400000070563
:101ED0000502400000070506024000000705070252
:101EE0004000000705810240000007058202400013
:101EF0000007058302400000070584024000000738
:101F0000058502400000070586024000000705879E
:101F100002400000040309042A034D006900630025
:101F200072006F00630068006900700020005400B8
:101F30006500630068006E006F006C006F00670052
:101F4000790020034900430044003200200055007E
:101F500053004200200044006500760069006300E1
:101F60006500120369006300640032002000750000
:101F700073006200A01EA01E141F181F421F621FC4
:101F80003816000EF66E010EF76E000EF86E0001A8
:101F90000900F550556F0900F550566F03E155677C
:101FA00001D03DD00900F550506F0900F550516F38
:101FB0000900F550526F09000900F550E96E09005B
:101FC000F550EA6E090009000900F550536F090049
:101FD000F550546F09000900F6CF57F0F7CF58F0CD
:101FE000F8CF59F050C0F6FF51C0F7FF52C0F8FFCC
:101FF0000001535302E1545307E00900F550EE6E1F
:102000005307F8E25407F9D757C0F6FF58C0F7FF57
:1020100059C0F8FF00015507000E565BBFD71200EC
:10202000036A026A016A006A200EE76ED8900436DD
:1020300005360636073600360136023603360950B5
:10204000005C0A5001580B5002580C50035809E329
:102050000950005E0A50015A0B50025A0C50035AA4
:10206000042AE72EE4D71200D8CFE4FFE0CFE4FF44
:10207000E46EDACFE4FFE2CFDAFFE652D59EF294C7
:10208000150ED76EA00ED66ED58E0001702B000EE9
:10209000712372237323E552E5CFDAFFE550E5CFD4
:1020A000E0FFE5CFD8FF100017EE00F027EE00F0BC
:1020B000F86A0F9CC1EC0FF0C8EC00F0FDD71200DD
:1020C000E000D0009603F00556081A018608E808DB
:1020D000A60C140DFFFFFFFFFFFFFFFFFFFFFFFF39
:1020E000FFFFFFFFFFFFFFFFFFFFFFFFFFFFFFFF00
:1020F000FFFFFFFFFFFFFFFFFFFFFFFFFFFFFFFFF0
:10210000FFFFFFFFFFFFFFFFFFFFFFFFFFFFFFFFDF
:10211000FFFFFFFFFFFFFFFFFFFFFFFFFFFFFFFFCF
:10280000B2EF23F01200FFFF92EF23F01200FFFF60
:10281000FFFFFFFFFFFFFFFFFFFFFFFFFFFFFFFFC8
:10282000FFFFFFFFFFFFFFFFFFFFFFFFFFFFFFFFB8
:10283000FFFFFFFFFFFFFFFFFFFFFFFFFFFFFFFFA8
:10284000FFFFFFFFFFFFFFFFFFFFFFFFFFFFFFFF98
:10285000FFFFFFFFFFFFFFFFFFFFFFFFFFFFFFFF88
:10286000FFFFFFFFFFFFFFFFFFFFFFFFFFFFFFFF78
:10287000FFFFFFFFFFFFFFFFFFFFFFFFFFFFFFFF68
:10288000FFFFFFFFFFFFFFFFFFFFFFFFFFFFFFFF58
:10289000FFFFFFFFFFFFFFFFFFFFFFFFFFFFFFFF48
:1028A000FFFFFFFFFFFFFFFFFFFFFFFFFFFFFFFF38
:1028B000FFFFFFFFFFFFFFFFFFFFFFFFFFFFFFFF28
:1028C000FFFFFFFFFFFFFFFFFFFFFFFFFFFFFFFF18
:1028D0000201FFFFFFFFFFFFFFFFFFFFFFFFFFFF03
:1028E00002008C4700005A000000040000007C47F2
:1028F00000004000000010000000D9CFE6FFE1CF4B
:10290000D9FF020EE1268F0EDE6E000EDD6EDECFE9
:10291000E9FFDDCFEAFF000EEF6A010EEB6AD00E91
:10292000F66E280EF76E0900F5CF10F00800F5CF0F
:1029300011F0DECFE9FFDDCFEAFF020EE926000E3F
:10294000EA2210C0EEFF11C0EDFF8F0EE66E000E02
:10295000E66E7EEC1AF0E552E552F56E020EE15C91
:1029600002E2E16AE552E16EF550E552E7CFD9FFA8
:102970001200010EE66E5FEC1BF0E5523BEC1BF023
:10298000140E6F6E0001976B0001986B0001996B3C
:1029900080A802D04AEC1BF093EC1DF0AFEC1DF0C8
:1029A00000090BE0080EE66E400EE66E000EE66EC5
:1029B000DFEC14F0E552E552E552EAD71200D9CF28
:1029C000E6FFE1CFD9FF120EE66E7D0EE66E000E39
:1029D000E66E1BEC1AF0E552E552E552FC0EDB50B8
:1029E0000001D8807D551FE3FD0EDBCF12F0FE0EF7
:1029F000DBCF13F07D51020D1250F324E96E13501A
:102A0000F420EA6EEECF10F0EFCF11F07D0EE66EFF
:102A1000000EE66E04D011C0FAFF1050F96EFBDF15
:102A2000E552E55210D00001010E8F6F906B916B53
:102A3000926B936B946B8F0EE66E000EE66E7EECDF
:102A40001AF0E552E55200017D69E552E7CFD9FF62
:102A50001200D9CFE6FFE1CFD9FF0E0EE126FD0E21
:102A6000DBCFE9FFFE0EDBCFEAFF020EE926000E08
:102A7000EA22EECF04F0EECF05F0EECF06F0EFCF76
:102A800007F0400E096E0A6A0B6A0C6A6EEC23F0BE
:102A900004C0DEFF05C0DDFFFD0EDBCFE9FFFE0E4B
:102AA000DBCFEAFF020EE926000EEA22EECF04F0A9
:102AB000EECF05F0EECF06F0EFCF07F0400E096E37
:102AC0000A6A0B6A0C6A6EEC23F0020E00C0DBFF90
:102AD000FD0EDBCFE9FFFE0EDBCFEAFF020EE9269B
:102AE000000EEA22080EE926000EEA22030EEECFBF
:102AF000DBFF040EEECFDBFF050EEECFDBFF060E95
:102B0000EECFDBFF0B0EDB6A0C0EDB6A0D0EDB6A11
:102B1000070EDB6A080EDB6A070EDBCF10F0080E2B
:102B2000DBCF11F0DECF12F0DDCF13F01250105CCE
:102B30001350115848E2D950090FE66E000EDA2002
:102B4000E66ED950030FE96EDACFEAFFEECFE6FF6B
:102B5000EECFE6FFEECFE6FFEFCFE6FF400EE66EEC
:102B6000E66A800EE66E050EE66ED6EC1CF0F56E9B
:102B70000A0EE15EF550E76E0D0EE7CFDBFF090EA2
:102B8000DBCF10F00A0EDBCF11F0D9500B0FE96E3E
:102B9000DACFEAFF1050EE261150ED22090EDBCFFE
:102BA000E6FF000EE66EE66A47EC1AF0E552E552E3
:102BB000E5520D0EDB5001E006D0070EDB2A080EB1
:102BC00001E3DB2AA9D7020EDB5042E00D0EDB50F9
:102BD0003FE1D950090FE66E000EDA20E66ED950BB
:102BE000030FE96EDACFEAFFEECFE6FFEECFE6FFA6
:102BF000EECFE6FFEFCFE6FF020EDBCFE6FFE66AA1
:102C0000800EE66E050EE66ED6EC1CF0F56E0A0E32
:102C1000E15EF550E76E0D0EE7CFDBFF090EDBCF6F
:102C200010F00A0EDBCF11F0D9500B0FE96EDACF9E
:102C3000EAFF1050EE261150ED22090EDBCFE6FF21
:102C4000000EE66EE66A47EC1AF0E552E552E552F0
:102C50000D0EDB5007E100018F6B906B916B926B57
:102C6000936B0BD00001020E8F6F0B0EDBCF90F039
:102C70000C0EDBCF91F0926B936B906B916B926B20
:102C8000936B946B8F0EE66E000EE66E7EEC1AF080
:102C9000E552E552F56E0E0EE15C02E2E16AE552A4
:102CA000E16EF550E552E7CFD9FF1200D9CFE6FF2C
:102CB000E1CFD9FF0E0EE126FD0EDBCFE9FFFE0EC0
:102CC000DBCFEAFF020EE926000EEA22EECF04F087
:102CD000EECF05F0EECF06F0EFCF07F0400E096E15
:102CE0000A6A0B6A0C6A6EEC23F004C0DEFF05C0B2
:102CF000DDFFFD0EDBCFE9FFFE0EDBCFEAFF020EAC
:102D0000E926000EEA22EECF04F0EECF05F0EECF7A
:102D100006F0EFCF07F0400E096E0A6A0B6A0C6AE4
:102D20006EEC23F0020E00C0DBFFFD0EDBCFE9FFEF
:102D3000FE0EDBCFEAFF020EE926000EEA22080EA5
:102D4000E926000EEA22030EEECFDBFF040EEECFE3
:102D5000DBFF050EEECFDBFF060EEECFDBFF0B0E2B
:102D6000DB6A0C0EDB6A0D0EDB6A070EDB6A080EEF
:102D7000DB6A070EDBCF10F0080EDBCF11F0DECFE1
:102D800012F0DDCF13F01250105C135011584EE2C8
:102D9000E66AE66A010EE66EE7EC1AF0E552E552E5
:102DA000E552D950090FE66E000EDA20E66ED950D2
:102DB000030FE96EDACFEAFFEECFE6FFEECFE6FFD4
:102DC000EECFE6FFEFCFE6FF400EE66EE66A000EBE
:102DD000E66E050EE66E1BEC1CF0F56E0A0EE15E6B
:102DE000F550E76E0D0EE7CFDBFF090EDBCF10F0DD
:102DF0000A0EDBCF11F0D9500B0FE96EDACFEAFFE4
:102E00001050EE261150ED22E66A000EE66EE66ADC
:102E100012DBE552E552E5520D0EDB5001E006D023
:102E2000070EDB2A080E01E3DB2AA3D7020EDB50D4
:102E300047E00D0EDB5044E1E66AE66A010EE66EFD
:102E4000C6DBE552E552E552D950090FE66E000E99
:102E5000DA20E66ED950030FE96EDACFEAFFEECF43
:102E6000E6FFEECFE6FFEECFE6FFEFCFE6FF020E86
:102E7000DBCFE6FFE66A000EE66E050EE66E1BECA3
:102E80001CF0F56E0A0EE15EF550E76E0D0EE7CF11
:102E9000DBFF090EDBCF10F00A0EDBCF11F0D950AB
:102EA0000B0FE96EDACFEAFF1050EE261150ED223B
:102EB000E66A000EE66EE66ABEDAE552E552E552D3
:102EC0000D0EDB5007E100018F6B906B916B926BE5
:102ED000936B0BD00001010E8F6F0B0EDBCF90F0C8
:102EE0000C0EDBCF91F0926B936B946B8F0EE66EB2
:102EF000000EE66E03DBE552E552F56E0E0EE15C68
:102F000002E2E16AE552E16EF550E552E7CFD9FF02
:102F10001200D9CFE6FFE1CFD9FFF5EC1BF000019D
:102F20008F6B906B916B926B936B946B8F0EE66EC5
:102F3000000EE66EE3DAE552E552E552E7CFD9FF3F
:102F40001200D9CFE6FFE1CFD9FF020EE1268F0EA6
:102F5000DE6E000EDD6EF29E5CC0F6FF5DC0F7FF18
:102F60000900F5CF10F00800F5CF11F0DECFE9FF32
:102F7000DDCFEAFF10C0EEFF11C0EDFFF28E8F0E25
:102F8000E66E000EE66EBADAE552E552F56E020E16
:102F9000E15C02E2E16AE552E16EF550E552E7CF0D
:102FA000D9FF1200D9CFE6FFE1CFD9FF090EE12604
:102FB00000018F6BFD0EDBCFE9FFFE0EDBCFEAFFDA
:102FC000020EE926000EEA22EECF10F0EFCF11F04C
:102FD000010E101801E1115001E102D1020E10188A
:102FE00001E1115049E0105001E1115001E0F8D029
:102FF000FD0EDBCFE9FFFE0EDBCFEAFF020EE92676
:10300000000EEA22040EE926000EEA22EECF10F0AE
:10301000EFCF11F0060ED89011321032E804FBE128
:1030200010C0DEFF11C0DDFFD9CFE9FFDACFEAFF24
:10303000EE50ED101DE0DECFE6FFDDCFE6FFFD0E2A
:10304000DBCFE9FFFE0EDBCFEAFF020EE926000E22
:10305000EA22020EE926000EEA22EECFE6FFEFCFCB
:10306000E6FFF1EC21F0E552E552E552E55203D0DE
:103070000001040E8F6F5CD1FD0EDBCFE9FFFE0E69
:10308000DBCFEAFF020EE926000EEA22040EE92653
:10309000000EEA22EECF10F0EFCF11F0060E0F0B6C
:1030A00005E0D89011321032E806FBE1040E10C0A2
:1030B000DBFF050E11C0DBFFFD0EDBCFE9FFFE0ECF
:1030C000DBCFEAFF020EE926000EEA22040EE92613
:1030D000000EEA22EECF10F0EFCF11F00001116ADE
:1030E0003F0E1016080E10C0DBFFFD0EDBCFE9FF10
:1030F000FE0EDBCFEAFF020EE926000EEA22020EE8
:10310000E926000EEA22060EEECFDBFF070EEDCF1A
:10311000DBFF020EDB6A030EDB6A020EDBCF10F070
:10312000030EDBCF11F0040EDBCF12F0050EDBCF68
:1031300013F01250105C135011582EE2E66AE66A42
:10314000010EE66E44DAE552E552E552000EE66EF7
:10315000050EE66E060EDBCFE6FF070EDBCFE6FFC1
:1031600029EC22F0E552E552E552E552D950060F1E
:10317000E96EDACFEAFF400EEE26000EED22E66A97
:10318000E66EE66A58D9E552E552E552020EDB2AB0
:10319000030E01E3DB2AC1D7080EDB5020E0E66A0C
:1031A000E66A010EE66E13DAE552E552E552000ECC
:1031B000E66E050EE66E060EDBCFE6FF070EDBCFF2
:1031C000E6FF29EC22F0E552E552E552E552E66AC7
:1031D000000EE66EE66A2FD9E552E552E552A8D018
:1031E000FD0EDBCFE9FFFE0EDBCFEAFF020EE92684
:1031F000000EEA22040EE926000EEA22EECF10F0BD
:10320000EFCF11F0060E0F0B05E0D89011321032FF
:10321000E806FBE1040E10C0DBFF050E11C0DBFF6A
:10322000FD0EDBCFE9FFFE0EDBCFEAFF020EE92643
:10323000000EEA22040EE926000EEA22EECF10F07C
:10324000EFCF11F00001116A3F0E1016080E10C0EA
:10325000DBFFFD0EDBCFE9FFFE0EDBCFEAFF020E48
:10326000E926000EEA22020EE926000EEA22060EE8
:10327000EECFDBFF070EEDCFDBFF020EDB6A030EA6
:10328000DB6A020EDBCF10F0030EDBCF11F0040E71
:10329000DBCF12F0050EDBCF13F01250105C135091
:1032A000115828E2800EE66E050EE66E060EDBCFA4
:1032B000E6FF070EDBCFE6FF7FEC22F0E552E5529A
:1032C000E552E552D950060FE96EDACFEAFF400E1B
:1032D000EE26000EED22400EE66E000EE66EE66A69
:1032E000D6D8E552E552E552020EDB2A030E01E381
:1032F000DB2AC7D7080EDB501AE0800EE66E050EFB
:10330000E66E060EDBCFE6FF070EDBCFE6FF7FECB7
:1033100022F0E552E552E552E552080EDBCFE6FF1A
:10332000000EE66EE66AB3D8E552E552E55200D0EB
:103330000001906B916B926B936B946B8F0EE66EAA
:10334000000EE66EDBD8E552E552F56E090EE15C43
:1033500002E2E16AE552E16EF550E552E7CFD9FFAE
:103360001200D9CFE6FFE1CFD9FF00018F6B906B40
:10337000916B926B936B946B8F0EE66E000EE66E04
:10338000BDD8E552E552C80EE66EE66AE66AE66A20
:10339000A7EC1BF0E552E552E552E5526D96F29E20
:1033A0005AC0F6FF5BC0F7FF020EF626000EF722AA
:1033B0000900F5CF10F00800F5CF11F004D011C0CE
:1033C000FAFF1050F96EFBDFE552E7CFD9FF12008C
:1033D000D9CFE6FFE1CFD9FF00018F6B906B916BE6
:1033E000926B936B946B8F0EE66E000EE66E86D832
:1033F000E552E552C80EE66EE66AE66AE66AA7ECB2
:103400001BF0E552E552E552E5526D96F29E5AC028
:10341000F6FF5BC0F7FF0900F5CF10F00800F5CF0D
:1034200011F004D011C0FAFF1050F96EFBDFE55225
:10343000E7CFD9FF1200D9CFE6FFE1CFD9FFD950AE
:10344000FD0FE96EFF0EDA20EA6EEE50ED1013E08C
:10345000FC0EDBCFE6FFE66A000EE66E050EE66EBA
:10346000FD0EDBCFE6FFFE0EDBCFE6FFD8D8F56E14
:10347000060EE15EF55068960401400E096F0817CC
:10348000087D880E0813E552E7CFD9FF1200D9CF87
:10349000E6FFE1CFD9FFD950FD0FE96EFF0EDA202C
:1034A000EA6EEE50ED1013E0FC0EDBCFE6FFE66AAD
:1034B000FD0EDBCFE6FFFE0EDBCFE6FF800EE66EF5
:1034C000050EE66EACD8F56E060EE15EF550FC0E0C
:1034D000DBCF15F4400E04011417147D880E14136D
:1034E000010EE66E040EE66E020EE66E70D8E55230
:1034F000E552E552E552E7CFD9FF1200D9CFE6FFFA
:10350000E1CFD9FF050EE1260EC4DEFF0FC4DDFFBB
:10351000FD0EDBCF06F0FE0EDBCF07F0020E06C07D
:10352000DBFF030E07C0DBFF080EF36E040EF3CFC4
:10353000DBFFDBCF0DF4DFCFE9FFDF2A010EDBCFAE
:10354000EAFF01E3DB2A7DC0EFFFDFCFE9FFDF2ADF
:10355000DBCFEAFF01E3DB2AEF6A040EDBCFF3FFE8
:10356000DB06F350000917E0020EDBCFE9FFDB2A90
:10357000030EDBCFEAFF01E3DB2AEF50E66EDFCF7D
:10358000E9FFDF2A010EDBCFEAFF01E3DB2AE55288
:10359000E750EF6EE2D7400E04010C170C7D880E49
:1035A0000C13010EE66E040EE66E010EE66E0FD8E9
:1035B000E552E552E552F56E050EE15C02E2E16A84
:1035C000E552E16EF550E552E7CFD9FF1200D9CFB1
:1035D000E6FFE1CFD9FF93EC1DF0AFEC1DF0000941
:1035E00019E0780E00017C15E840E840E8401F0B28
:1035F000106EFE0EDB50105C0DE1040E7C15116E9A
:10360000FD0EDB50115C06E1FC0EDB5001E068961C
:1036100002D000D0E0D7E552E7CFD9FF1200D9CFD2
:10362000E6FFE1CFD9FFF90EDBCF10F0DB06FA0E93
:10363000DBCF11F001E2DB061050111018E0FB0E99
:10364000DBCFE9FFDB2AFC0EDBCFEAFF01E3DB2A5D
:10365000EF50E66EFD0EDBCFE9FFDB2AFE0EDBCF7F
:10366000EAFF01E3DB2AE552E750EF6EDCD7E552D3
:10367000E7CFD9FF12000F0EC16E070EB46E8B8418
:1036800094948B92949280807E0E926EE7EF1BF062
:103690006D96120019EC1CF0FBDF8BA202D08B920E
:1036A00001D08B82140EE66EE66AE66AE66AA7EC43
:1036B0001BF0E552E552E552E552EFD71200D9CFA3
:1036C000E6FFE1CFD9FF0001706B716B726B736B1A
:1036D000D56AD08EFE0EDB5002E0F18401D0F19469
:1036E000150ED76EA00ED66EF294F28AF28CF28E80
:1036F000D58EE552E7CFD9FF1200D9CFE6FFE1CF53
:10370000D9FF040EE126F29A70C0DFFF010E71C0EE
:10371000DBFF020E72C0DBFF030E73C0DBFFF28A19
:10372000DECF04F0DECF05F0DECF06F0DDCF07F010
:10373000DD52DD52F56E040EE15C03E200D0E16A79
:10374000E552E16EF550E552E7CFD9FF1200D9CF2F
:10375000E6FFE1CFD9FF040EE12670C0DFFF010EC6
:1037600071C0DBFF020E72C0DBFF030E73C0DBFF14
:10377000FB0EDBCF10F0FC0EDBCF11F0FD0EDBCF2C
:1037800012F0FE0EDBCF13F0D9CFE9FFDACFEAFF5C
:10379000EE501026EE501122EE501222EE5013225F
:1037A00010500001705D1150715912507259135030
:1037B000735901E2DDD7F56E040EE15C02E2E16AC5
:1037C000E552E16EF550E552E7CFD9FF1200F18ED8
:1037D000470E836E956A8A888D808D828A96E70E61
:1037E000936EF90E946E966A1200D9CFE6FFE1CF80
:1037F000D9FF020EE1268A86DE6ADD6ADECF10F08E
:10380000DDCF11F0480E105C920E115805E2DF2A50
:10381000010E01E3DB2AF2D78A96F56E020EE15C17
:1038200002E2E16AE552E16EF550E552E7CFD9FFD9
:1038300012008A861200D9CFE6FFE1CFD9FF070E2A
:10384000E126DF6AD950F70FE96EFF0EDA20EA6E43
:10385000050EEE5C000EEE58000EEE58000EEE580F
:103860000BE2050EF36EF70EF3CFDBFFF80EDB6A0B
:10387000F90EDB6AFA0EDB6A050EDB6A060EDB6AFE
:10388000050EDBCF10F0060EDBCF11F0FB0EDBCF09
:1038900012F0FC0EDBCF13F01250105C13501158D5
:1038A0006BE27DEC1BF0010E04C0DBFF020E05C0D5
:1038B000DBFF030E06C0DBFF040E07C0DBFF82B098
:1038C00042D0010EDBCF14F0020EDBCF15F0030E59
:1038D000DBCF16F0040EDBCF17F014C0E6FF15C0E7
:1038E000E6FF16C0E6FF17C0E6FF7DEC1BF0E552D1
:1038F000E7CF17F0E552E7CF16F0E552E7CF15F026
:10390000E552E7CF14F000011450045C106E15501E
:103910000558116E16500658126E17500758136E40
:10392000D950F70FE96EFF0EDA20EA6E1050EE5C08
:103930001150EE581250EE581350EE5803E2010E9B
:10394000DF6E01D0BCD7DF0402E116D00FD08A9819
:103950008D90FD0EDBCFE9FFDB2AFE0EDBCFEAFF09
:1039600001E3DB2AEF50836E8D808A88050EDB2A07
:10397000060E01E3DB2A84D7F50EDBCFE9FFF60E56
:10398000DBCFEAFF050EDBCFEEFF060EDBCFEDFF50
:10399000DF50F56E070EE15C03E200D0E16AE5520C
:1039A000E16EF550E552E7CFD9FF1200D9CFE6FF1F
:1039B000E1CFD9FF070EE126DF6AD950F70FE96E94
:1039C000FF0EDA20EA6E050EEE5C000EEE58000ED9
:1039D000EE58000EEE580BE2050EF36EF70EF3CF25
:1039E000DBFFF80EDB6AF90EDB6AFA0EDB6A050E06
:1039F000DB6A060EDB6A050EDBCF10F0060EDBCFAE
:103A000011F0FB0EDBCF12F0FC0EDBCF13F01250E7
:103A1000105C135011586DE27DEC1BF0010E04C0D8
:103A2000DBFF020E05C0DBFF030E06C0DBFF040E4A
:103A300007C0DBFF82B042D0010EDBCF14F0020ED4
:103A4000DBCF15F0030EDBCF16F0040EDBCF17F043
:103A500014C0E6FF15C0E6FF16C0E6FF17C0E6FF7C
:103A60007DEC1BF0E552E7CF17F0E552E7CF16F0FB
:103A7000E552E7CF15F0E552E7CF14F000011450FE
:103A8000045C106E15500558116E16500658126ED3
:103A900017500758136ED950F70FE96EFF0EDA2052
:103AA000EA6E1050EE5C1150EE581250EE58135062
:103AB000EE5803E2010EDF6E01D0BCD7DF0402E155
:103AC00018D011D095688A988D928D82FD0EDBCF2B
:103AD000E9FFDB2AFE0EDBCFEAFF01E3DB2A83CF1F
:103AE000EFFF8A88956A050EDB2A060E01E3DB2AC2
:103AF00082D7F50EDBCFE9FFF60EDBCFEAFF050E2E
:103B0000DBCFEEFF060EDBCFEDFFDF50F56E070ECD
:103B1000E15C03E200D0E16AE552E16EF550E55266
:103B2000E7CFD9FF12006DA60CD80001970508E178
:103B30006DBA06D0686A696A69806988020E976FF3
:103B400012006D6A696A6D860001010E976F12009E
:103B50006D6A696A0001976B1200A8EF1DF0D9CF5A
:103B6000E6FFE1CFD9FF020EE126010EDB6A00017C
:103B7000975101E152D06850040B04E06950040BE6
:103B800001E05ED86DB249D06850010B04E0695085
:103B9000010B01E078D86850100B04E06950100B5D
:103BA00001E04AD86850400B04E06950400B01E046
:103BB0005DD86850200B04E06950200B01E058D814
:103BC0006850020B04E06950020B01E05AD8030E62
:103BD0000001975D01E221D06850080B1CE069509C
:103BE000080B19E0F1EC1EF0F3CF10F0F4CF11F058
:103BF000105011100FE16C50DF6EDFCF7CF0780EAB
:103C0000DF14E840E840E8401F0BE76E010EE7CF05
:103C1000DBFF01D0689601D0AAD7010EDB50F56E0C
:103C2000020EE15C03E200D0E16AE552E16EF5507C
:103C3000E552E7CFD9FF1200698468986D821200BF
:103C40006D92699468941200000198A10ED0F8DF7B
:103C50006D840001080E956F070E966F9507000E94
:103C6000965B95519611FAE16D941200689C1200D2
:103C7000010E7014010803E15FEC20F07090689A67
:103C80001200689212006A6A686A9F0E6B6E7B0E61
:103C9000696E6E6A0F0EE66E710EE66E0F0EE66EC0
:103CA00014D8E552E552E552160E706E68A602D0A1
:103CB0006896FCD76D985FEC20F0000198910001A8
:103CC000996B0001030E976F1200D9CFE6FFE1CF89
:103CD000D9FFFD0EDBCFE9FFFE0EDBCFEAFFFC0EC6
:103CE000DB5004E0EE6AFC0EDB06F9D7E552E7CFC5
:103CF000D9FF1200040140511F0B010801E011D04F
:103D00004051600BE842E842E842E842E8420208DB
:103D100001E007D0445101E004D0415101E001D05D
:103D200000D0120000017D690401400E096F000EF1
:103D30000A6F050E0B6F800E086F0401400E0D6FA9
:103D4000400E0E6F050E0F6F400E0C6F0401126BCC
:103D5000136B800E106F0401400E156F800E166FEE
:103D6000050E176F400E146F04011A6B1B6B800E4B
:103D7000186F04011E6B1F6B400E1C6F0401226B39
:103D8000236B800E206F0401266B276B400E246F7F
:103D900004012A6B2B6B800E286F04012E6B2F6B96
:103DA000400E2C6F0401326B336B800E306F0401B8
:103DB000366B376B400E346F04013A6B3B6B800EF1
:103DC000386F04013E6B3F6B400E3C6F1E0E716EF0
:103DD0001A0E726E180E736E746E756E766E776E46
:103DE0001200D9CFE6FFE1CFD9FF020EE126010E86
:103DF000DE6EDD6A6C500BE1040100513C0BE842C1
:103E0000E8420D0802E11FD801D031D807D0040ED6
:103E10006C5C02E13CD802D0DE6ADD6ADECF10F0D5
:103E2000DDCF11F010C0F3FF11C0F4FFF56E020EEC
:103E3000E15C03E200D0E16AE552E16EF550E55243
:103E4000E7CFD9FF1200D9CFE6FFE1CFD9FFE65285
:103E50000001746B0001756B00017A6B7B6B6DEC7C
:103E600020F0E7D8E552E552E7CFD9FF1200020E65
:103E70000001745D0AE19BD8040100BD03D0C80EA7
:103E8000006F02D0880E006F01D019D91200040E05
:103E90000001975D0AE142C46EFF6E50000803E224
:103EA000050E976F02D0030E976F000174050AE1AB
:103EB0000BD8040104BD03D0C80E046F02D0880ED5
:103EC000046F01D0FCD81200D9CFE6FFE1CFD9FFB3
:103ED000020EE1260001080E7A5D000E7B5905E214
:103EE0007AC0DEFF7BC0DDFF03D0080EDE6EDD6A28
:103EF000040104930491010EDB500413DFCF05F499
:103F0000000EDB5000017A5F010EDB507B5B00018D
:103F1000480E786F040E796F000198A31FD0D9CF97
:103F2000E9FFDACFEAFFEE50ED1017E076C0F6FFBA
:103F300077C0F7FF0800F55078C0E9FF79C0EAFFC5
:103F4000EF6E0001782B000E79230001762B77238A
:103F5000DF06010E01E2DB06E2D71DD0D9CFE9FF73
:103F6000DACFEAFFEE50ED1016E076C0E9FF77C039
:103F7000EAFFEF5078C0E9FF79C0EAFFEF6E000179
:103F8000782B000E79230001762B7723DF06010EB4
:103F900001E2DB06E3D7F56E020EE15C02E2E16AC4
:103FA000E552E16EF550E552E7CFD9FF1200D9CFC7
:103FB000E6FFE1CFD9FF020EE126030E0401001552
:103FC000E76E010EE7CFDBFF01C4DFFFDE5000012B
:103FD0007A27DD507B230001480E766F040E776F41
:103FE000D9CFE9FFDACFEAFFEE50ED1016E076C048
:103FF000E9FF77C0EAFFEF5078C0E9FF79C0EAFF38
:10400000EF6E0001782B000E79230001762B7723C9
:10401000DF06010E01E2DB06E3D7F56E020EE15C7E
:1040200002E2E16AE552E16EF550E552E7CFD9FFD1
:104030001200000175510CE10401080E016F400EE1
:10404000026F040E036F840E006F0401046F35D0FD
:10405000040140AF22D000017A510401465D000105
:104060007B510401475904E246C47AF047C47BF00F
:104070002BDF0001010E746F0401080E016F400E6A
:10408000026F040E036F800E006F0401480E066F6E
:10409000040E076FC80E046F10D00001020E746F7B
:1040A0000401056BC80E046F0401080E016F480E71
:1040B000026F040E036FC80E006F6D9812000001AE
:1040C000746B0401080E016F400E026F040E036F43
:1040D000880E006F0401046B120004014051600B54
:1040E000E842E842E842E842E842000901E055D0EF
:1040F0004151070A51E00B0A4FE0070A40E0010A6C
:104100002CE00B0A28E0020A26E0030A22E0080A53
:1041100012E0010A0EE00F0A0AE0030A01E03CD0B7
:104120000001010E756F0001040E976F36D036D86E
:1041300034D090D832D00001010E756F0001990E75
:10414000766F000E776F000198930001010E7A6F71
:1041500024D0A8D822D0F4D820D00001010E756F49
:10416000040144510001766F776B9A0E7627000E9A
:104170007723000198930001010E7A6F0ED00001A1
:10418000010E756F04014451EA6A9A0FE96E000E40
:10419000EA2242C4EFFF01D000D01200800E0401D9
:1041A000405D57E14351030A34E0010A10E0030A7D
:1041B00001E04DD00001010E756F00014A0E766FCF
:1041C000450E776F120E00017A6F7B6B40D00001B5
:1041D000010E756F04014251F66EF76AD890F636FB
:1041E000F736300EF626460EF7220900F5CF76F0A8
:1041F0000A00F5CF77F0020E0001F76A7625F66E19
:104200007751F7220900F5CF7AF00A00F5CF7BF05D
:104210001ED00001010E756F04014251F66EF76A5F
:10422000D890F636F736340EF626460EF7220900F9
:10423000F5CF76F00A00F5CF77F076C0F6FF77C0BD
:10424000F7FF0800F55000017A6F7B6B00D000018A
:10425000988312000001010E756F0F0EE66E710E4D
:10426000E66E0F0EE66E65EC1EF0E552E552E55285
:10427000010EE66E9A0EE66E000EE66E65EC1EF01E
:10428000E552E552E55242C499F00401425104E17D
:104290000001050E976F05D00001060E976F92EC96
:1042A0001EF012000401486B496B040140511F0BC2
:1042B000020A14E0030A0EE0010A01E033D0000113
:1042C000010E756F04014881000198A102D004011C
:1042D000488328D00001010E756F24D00001010E23
:1042E000756F040144510F0B080DF350116A000F54
:1042F000106E040E11224451800B01E0010E040DDA
:10430000F35000011024786F000E1120796F78C0EF
:10431000E9FF79C0EAFFEF50040B03E00401010E4E
:10432000486F00D0000175050AE10001480E766F64
:10433000040E776F000198930001020E7A6F12004D
:104340000401420510E140511F0B00090CE100017E
:10435000010E756F030E0401415D03E100019881B8
:1043600002D000019891040142513AE140511F0BE3
:10437000020836E144510F0B000932E00001010E42
:10438000756F040144510F0B080DF350116A000FB3
:10439000106E040E11224451800B01E0010E040D39
:1043A000F35000011024786F000E1120796F030E76
:1043B0000401415D07E1840E78C0E9FF79C0EAFF9E
:1043C000EF6E0ED044AF06D078C0E9FF79C0EAFFA7
:1043D000EF6A06D0880E78C0E9FF79C0EAFFEF6E79
:1043E0001200D9CFE6FFE1CFD9FFFD0EDBCFF6FFFC
:1043F000FE0EDBCFF7FFF86AA68EA69CA684A688E1
:10440000F29E550EA76EAA0EA76EA6820000A6B257
:1044100007EF22F0F28EA694FB0EDB06FC0E01E203
:10442000DB06D950FB0FE96EFF0EDA20EA6EEE5084
:10443000ED100BE0D950FD0FE96EFF0EDA20EA6EA9
:10444000400EEE26000EED22D0D7E552E7CFD9FF81
:104450001200D9CFE6FFE1CFD9FF020EE126DE52EE
:10446000020EDD6EFD0EDBCFF6FFFE0EDBCFF7FF9B
:10447000F86A200EDF6EFB0EDBCFE9FFDB2AFC0EB5
:10448000DBCFEAFF01E3DB2AEF50F56E0D00DF061C
:10449000DF50000801E2EFD7FD0EDBCFF6FFFE0E86
:1044A000DBCFF7FFF86AA68EA69CA684A698F29E9C
:1044B000550EA76EAA0EA76EA6820000A6B25EEFEA
:1044C00022F0F28EA694010EDB06010EDB500BE00B
:1044D000D950FD0FE96EFF0EDA20EA6E200EEE26AF
:1044E000000EED22BFD7F56E020EE15C02E2E16A3A
:1044F000E552E16EF550E552E7CFD9FF1200D9CF72
:10450000E6FFE1CFD9FFE652400EDF6EFD0EDBCFB6
:10451000F6FFFE0EDBCFF7FFF86A0900FB0EDBCFDC
:10452000E9FFFC0EDBCFEAFFF5CFEFFFFB0EDB2A46
:10453000FC0E01E3DB2ADF06DF50000801E2EDD7C5
:10454000E552E552E7CFD9FF120012010001FFFF4B
:10455000FF08D80401801000000000010902740067
:104560000101008032090400000EFFFFFF00070573
:104570000102400000070502024000000705030297
:104580004000000705040240000007050502400046
:10459000000705060240000007050702400000076B
:1045A00005810240000007058202400000070583E4
:1045B0000240000007058402400000070585024014
:1045C0000000070586024000000705870240000042
:1045D000040309042A034D006900630072006F00A0
:1045E00063006800690070002000540065006300EB
:1045F00068006E006F006C006F0067007900200398
:10460000490043004400320020005500530042009E
:104610002000440065007600690063006500120315
:1046200069006300640032002000750073006200BE
:104630005C455C45D045D445FE451E46F43CE00E45
:10464000F66E280EF76E000EF86E00010900F550A8
:10465000556F0900F550566F03E1556701D03DD005
:104660000900F550506F0900F550516F0900F550E1
:10467000526F09000900F550E96E0900F550EA6E25
:10468000090009000900F550536F0900F550546FF7
:1046900009000900F6CF57F0F7CF58F0F8CF59F0DE
:1046A00050C0F6FF51C0F7FF52C0F8FF000153534E
:1046B00002E1545307E00900F550EE6E5307F8E2AB
:1046C0005407F9D757C0F6FF58C0F7FF59C0F8FF95
:1046D00000015507000E565BBFD71200036A026A3D
:1046E000016A006A200EE76ED89004360536063659
:1046F000073600360136023603360950005C0A5090
:1047000001580B5002580C50035809E30950005E41
:104710000A50015A0B50025A0C50035A042AE72E31
:10472000E4D71200D8CFE4FFE0CFE4FFE46EDACFA5
:10473000E4FFE2CFDAFFE652D59EF294150ED76E73
:10474000A00ED66ED58E0001702B000E7123722341
:104750007323E552E5CFDAFFE550E5CFE0FFE5CF83
:10476000D8FF100017EE00F027EE00F0F86A0F9C5B
:104770001FEC23F0B9EC14F0FDD71200522AAC2C38
:10478000122FFA28422FA42F6233D033E000D0003A
:10479000FFFFFFFFFFFFFFFFFFFFFFFFFFFFFFFF29
:1047A000FFFFFFFFFFFFFFFFFFFFFFFFFFFFFFFF19
:1047B000FFFFFFFFFFFFFFFFFFFFFFFFFFFFFFFF09
:1047C000FFFFFFFFFFFFFFFFFFFFFFFFFFFFFFFFF9
:107FF000FFFFFFFFFFFFFFFFFFFFFFFFFFFFE1E4CA
:0200000400F00A
:10000000FFFFFFFFFFFFFFFFFFFFFFFFFFFFFFFF00
:10001000FFFFFFFFFFFFFFFFFFFFFFFFFFFFFFFFF0
:10002000FFFFFFFFFFFFFFFFFFFFFFFFFFFFFFFFE0
:10003000FFFFFFFFFFFFFFFFFFFFFFFFFFFFFFFFD0
:10004000FFFFFFFFFFFFFFFFFFFFFFFFFFFFFFFFC0
:10005000FFFFFFFFFFFFFFFFFFFFFFFFFFFFFFFFB0
:10006000FFFFFFFFFFFFFFFFFFFFFFFFFFFFFFFFA0
:10007000FFFFFFFFFFFFFFFFFFFFFFFFFFFFFFFF90
:10008000FFFFFFFFFFFFFFFFFFFFFFFFFFFFFFFF80
:10009000FFFFFFFFFFFFFFFFFFFFFFFFFFFFFFFF70
:1000A000FFFFFFFFFFFFFFFFFFFFFFFFFFFFFFFF60
:1000B000FFFFFFFFFFFFFFFFFFFFFFFFFFFFFFFF50
:1000C000FFFFFFFFFFFFFFFFFFFFFFFFFFFFFFFF40
:1000D000FFFFFFFFFFFFFFFFFFFFFFFFFFFFFFFF30
:1000E000FFFFFFFFFFFFFFFFFFFFFFFFFFFFFFFF20
:1000F000FFFFFFFFFFFFFFFFFFFFFFFFFFFFFFFF10
:020000040030CA
:0E000000240F3900008180000FC00FE00F4078
:020000040020DA
:08000000FFFFFFFFFFFFFFFF00
:00000001FF
